:020000040000FA
:0400000064009A28D6
:0800080064009400030893005A
:100010000B1D25280B119A0B40289C08031D9C03DF
:100020009B08031D9B039808031D98039908031D53
:1000300099039D0B23283C309D009E08031D9E03C1
:100040009F08031D9F03FA309A008B1C40288B10D9
:100050000408A9000D08AA000C08AB008D018C0152
:1000600048202C0884000E088000AC0A2C08323C82
:10007000031945282A088D002B088C0029088400C4
:1000800013088300940E140E09002E30AC003A2899
:1000900086100D0851208F000C0851208E00861408
:1000A0000800900008309200900D06120318061602
:1000B0000615031086190314910D0611920B54288E
:1000C00011080800950064008D010D178C0148206F
:1000D0000F1F632815088C0080308D004820080011
:1000E0001F39803E622008000F3940386220080026
:1000F0009600023095289600083095289600013029
:10010000952896000930952896000D309528960080
:100110000E30952896000C309528960012309528C0
:100120009600103095289600113070201608742023
:100130001608080083161F308500E93086008312F8
:10014000051E0028850186012E30AC00AD0001306F
:100150009E009B00A201A10199019701E4308D004E
:1001600002308C00482040308D008C0148200E0861
:10017000023C031DAE288316833081008312303089
:100180008B008B17F0306220F7306220F530622050
:10019000FD306220FF306220043099009908031D71
:1001A000CE2803018A2003018420030178200A302D
:1001B0009020061FDB280130861F03308720FB308C
:0E01C0006220980199019F010A148A100029FB
:100200006400051E00281808013C03195421190830
:10021000013C03195B211F08013C031958212C08DC
:100220002D02031930292D080B128400AD0A2D0868
:10023000323C031D1D292E30AD0000080F39A300EC
:1002400000080B16F039A500A50E0310250C820737
:1002500069293029662930296B29712930296A29B1
:100260009B08031D3B29A80AA811861FA81528086A
:1002700084201E309B001E08013C031D00294121E3
:1002800000290B309E00261D47290F3087200030A3
:10029000861F02308720261D08000130861F05308A
:1002A0008A20083098000800980103018A2008007D
:1002B0009F01030190200230261D003078207E200F
:1002C0000730261D03307B20812008000A108A1485
:1002D000002A002900292608F039A6002308A604D0
:1002E000862926080F39A600230EA604171C80298C
:1002F0002619862917100D30872003018D208629A5
:10030000261D862917140E3087209F019F08031D84
:1003100000299908031D00290230261D003078208D
:100320007E200730261D03307B20812001309E0077
:020330000029A2
:10040000261D1C2A2308B822A0000E3C031D0C2A1E
:10041000A20106309C001C2A9C0803191A2AA20A71
:100420002208073982071A2A1F2A2A2A2D2A302A47
:100430001A2A1A2AA2019C010A148A1000292008EB
:10044000861F262A013C031D1A2A1C2A023C031D72
:100450001A2A1C2A200EA1001C2A2008A1041C2AEA
:1004600020080F3C031D1A2A9C0803191A2A9C0114
:10047000A201210E0F398207522A1A2A1A2A1A2A91
:100480001A2A1A2A872A562A602A742A1A2A1A2A03
:100490001A2A4C2A1A2A1A2A2108DC3C031D1A2A75
:1004A0008B13512A21080F398D201A2A20309F00E2
:1004B0000430782002307B2021080F3990201A2A3E
:1004C0002108823C031D692A0030861F02308720E4
:1004D0001A2A2108813C031D1A2A0130861F053083
:1004E0008A20083098001A2A2108993C031D1A2AEC
:1004F00099019F010230261D003078207E200730B0
:10050000261D03307B208120030190201A2A210818
:100510000739A1009D22260503191A2A2108A622BF
:1005200078207E202108AF227B2081200301211822
:1005300001309320783099001A2A82070834083451
:1005400010342034403480340234043482070334BD
:10055000033404340534063407340134003482078C
:1005600006340634023404340134033405340734C9
:1005700082070D3401340234033404340534063464
:1005800007340834093400340E340F340A340B3481
:020590000C3429
:02400E00F53F7C
:00000001FF
